:02000000682B6B
:020008000029CD
:10020000A600030EA7000B1930298B182029270EF2
:100210008300A60E260E09006400810183160313D5
:1002200088308100831286140614A50183160313F7
:1002300019309900243098008312903098000800FB
:100240008B100C30A000A00B232906180729AD3015
:10025000810020308B000230A5000830A000072963
:100260000B1125194329A00803193C29060CA10CE0
:10027000A003AD3081000729061C59290130A500D3
:100280002108A2005929A5195929A00803195129A3
:10029000A30C031C861003188614A003B53081003C
:1002A00007290000000000008614A515A830810071
:1002B000072900308B000130A50507296400A80B31
:1002C0006E29A90B1F2C0130AA06031D69290714EA
:1002D0006A2907100030A8001830A9003030050541
:1002E000B1003202031D80210C300505B9003A022D
:1002F000031DAA213108B2003908BA00D629080026
:1003000032083106303C0319D429310DB206B21E31
:100310009A2941189C29AD08031D9829AE08031D90
:1003200097292B08AD002C08AE00AD080319AE03C9
:10033000AD03080041188B29AD0A0319AE0A2B083A
:100340002D02031D08002C082E02031D0800AD011C
:10035000AE0108003A0839060C3C0319D429390DBE
:10036000BA06BA1DC4294218C629B508031DC229F8
:10037000B608031DC1293308B5003408B600B50816
:100380000319B603B50308004218B529B50A0319C5
:10039000B60A33083502031D080034083602031D6F
:1003A0000800B501B6010800BB0A08006400050892
:1003B000033946050319032AC3080319032AC5088C
:1003C0000319032A87118716FF30C70000000000B9
:1003D00000000000000000000000000000006400B9
:1003E000C70BE6298712FF30C7000000000000009D
:1003F0000000000000000000000000006400C70BC7
:10040000F529C50308008715C301080087145E217C
:100410008C1E072A9818122A181D142A181218164A
:100420001A080800181218161A08A20087100800E7
:10043000A3005E210C1E192A2308990007115E21D2
:100440000C1E1F2A0715080088223F08B3003E082B
:10045000B40088223F08AB003E08AC003322523083
:100460001822B723A52B8312031700308D002B0809
:100470008C006B228312031701308D002C088C0036
:100480006B228312031702308D0033088C006B221D
:100490008312031703308D0034088C006B2A8312FB
:1004A000031704308D0041088C006B2A8312031758
:1004B00005308D0042088C006B2A8312031706302A
:1004C0008D005E088C006B2A8312031707308D00A5
:1004D0005F088C006B2A6400831603130D168312C9
:1004E00003130D128B130B17831603178C130C15A4
:1004F00055308D00AA308D008C1463000C118316CA
:1005000003130D12831203130D120B138B17080024
:1005100063308400A401BF01BE01A408031D9E2A0C
:1005200006222208203C03198D2A22080D3C0319BB
:100530008D2A22088000A40A840A902A84030030AD
:10054000BC000130BD00C822A40BA72A0800840308
:100550000030BC000A30BD00C822A40BB02A08003D
:1005600084030030BC006430BD00C822A40BB92A4B
:10057000080084030330BC00E830BD00C822A40B8F
:10058000C22A080084032730BC001030BD00C82AEE
:100590002F300002C000C00BCE2A08003D08BF0764
:1005A0000318BE0A3C08BE07CB2A3B08BD00BC01AD
:1005B0004523203018224108303E182220301822CE
:1005C0004208303E1822203018220508BD00BC0128
:1005D0004523B723BB01A52B2D08AF002E08B00083
:1005E0003508B7003608B8003708BD003808BC0029
:1005F0000223093018222F08BD003008BC00022356
:10060000B723A52B2B301822372B88223F08C10097
:100610004F22443018223F08303E1822B723A52B22
:1006200088223F08C2005622523018223F08303E2E
:100630001822B723A52B88223F08B5003E08B60034
:1006400088223F08AD003E08AE0053301822B72381
:10065000A52B3408BC003308BD00372320301822F6
:100660002C08BC002B08BD003723B723A52B27304F
:10067000BE001030BF005623400818220330BE00D1
:10068000E830BF005623400818220030BE00643016
:10069000BF005623400818220030BE000A30BF00B9
:1006A0005623400818223D08303E182A2F30C0003B
:1006B000C00A3F08BD023E08031C013EBC020318ED
:1006C000582B3F08BD073E080318013EBC07080031
:1006D000831203138501831606309F00FF308500C7
:1006E000FD308600C0308700831203130712071401
:1006F0000030AA00A8001830A90087140715871534
:10070000871230300505B2000C300505BA00C5016E
:10071000C3010830C8000130C6000C21BB230030E3
:100720008B00FF30D000CF00CE00CD00CC00CB003E
:10073000CA00C900D100D500D400D300D200D60031
:100740000130D7000030D800D900062207308A00D7
:10075000DA015A08C027FF390319A52B2202031911
:10076000B32BDA0AA92B07308A005A08C92F0D309B
:1007700018220A30182A64008312031700308D00F3
:10078000831603178C130C14831203170C08AB0089
:1007900001308D00831603178C130C14831203177A
:1007A0000C08AC0002308D00831603178C130C1458
:1007B000831203170C08B30003308D008316031750
:1007C0008C130C14831203170C08B40004308D0032
:1007D000831603178C130C14831203170C08C10023
:1007E00005308D00831603178C130C148312031726
:1007F0000C08C20006308D00831603178C130C14EE
:10080000831203170C08DE0007308D0083160317D0
:100810008C130C14831203170C08DF000313BB01A5
:100820003308B5003408B6000310B60CB50C2B081D
:10083000AD002C08AE000310AE0CAD0C0800640037
:100840004F08D0004E08CF004D08CE004C08CD0018
:100850004B08CC004A08CB004908CA000608C0393A
:10086000C90050084F044E044D044C044B044A0484
:100870004904D1003230C4005108C03C03195E2C39
:100880005208530454045504DA00DA1F7A2C5A1F14
:10089000742C480803194E2CC803702C5408D5003A
:1008A0005308D4005208D3005108D2004030C80089
:1008B0000130C400D11F772C511F712CFF30D000A4
:1008C000CF00CE00CD00CC00CB00CA00C900D100C3
:1008D000D500D400D300D2000830C8000030C500D5
:1008E0006E29C308031D702C0230C6007C2CC3087F
:1008F000031D702C0130C6004408C5000130C30040
:10090000702C7C30E1006400E10B832C0800E200D5
:080910008124E20B882C080091
:100F800082075134563476345334523448347134F1
:100F900000348207EC2A052B102B1B2B242A292B2B
:020FA000D52A50
:02400E00713F00
:104200000000200000002000000000000600060062
:00000001FF
